:020000040000FA
:1000000000880002210100001D0100001D01000008
:1000100000000000000000000000000000000000E0
:1000200000000000204B0000684B00001D01000094
:1000300000000000000000001D0100001D01000084
:100040001D0100001D0100001D0100001D01000038
:100050001D0100001D0100001D0100001D01000028
:100060001D0100001D0100001D0100001D01000018
:100070001D010000510100001D0100001D010000D4
:100080001D0100001D0100001D0100001D010000F8
:100090001D0100001D0100001D0100001D010000E8
:1000A0001D0100001D0100001D0100001D010000D8
:1000B0001D0100001D010000000000000000000004
:1000C0000348854600F018F8004800478101000009
:1000D0000088000203460B439B0703D009E008C9D0
:1000E000121F08C0042AFAD203E00B780370401CE8
:1000F000491C521EF9D27047064C0125064E05E0F8
:10010000E36807CC2B430C3C98471034B442F7D338
:10011000FFF7DAFFF04A0000004B0000FEE70000A6
:1001200006480168032291430160016801220A43E5
:10013000026000F005F800F043F8C04628000040D7
:100140000148024901607047008000020026B803A0
:1001500080B582B0002001902B48C268002A02D0EE
:1001600001A80021904702B080BDC0460121814016
:10017000024802688A4302607047C046200000407F
:1001800070B50024204600F01FF80A4D0A4E0B4AB5
:1001900028463146FFF79EFF01204006C022314627
:1001A000FFF798FF286880F3088868688047204632
:1001B00070BDC04600A0020238020000B84800002E
:1001C00000480047C1000000B0B5002801D0012060
:1001D000B0BD032081020C4802680C4B5350002430
:1001E0009460012253030A4D2B60BFF34F8FBFF37E
:1001F0006F8F084D2B6003685A5084720481102061
:10020000FFF7B4FF2046B0BD0480000251E5CC1AD0
:1002100080E100E080E200E002E008C8121F08C1AF
:10022000002AFAD170477047002001E001C1121F77
:10023000002AFBD1704700000000030235AC020227
:100240002DA302022DA30202000000000000000006
:1002500000000000000000000000000020E8020292
:1002600068E802022DA30202000000000000000066
:100270002DA3020221B3020283A102022DA30202D6
:100280002DA3020255AC02022DA302022DA30202ED
:10029000BDA202025DA302022DA302022DA302024F
:1002A0002DA3020231A302022DA30202A1B3020276
:1002B0002DA302022DA302022DA302022DA30202EE
:1002C0002DA3020249B3020269B302022DA3020266
:1002D0002DA302022DA302028DB3020297B30202E4
:1002E00085A102022DA302022DA302022DA3020268
:1002F00000000000000000000348854600F02EF8D2
:1003000000480047F5D702020000030230B50B4653
:10031000014600202022012409E00D46D5409D42DF
:1003200005D31D469540491B254695404019154665
:10033000521E002DF1DC30BD03460B439B0703D05A
:1003400009E008C9121F08C0042AFAD203E00B789A
:100350000370401C491C521EF9D27047064C0125FF
:10036000064E05E0E36807CC2B430C3C984710345D
:10037000B442F7D3FFF7C4FF14E6020234E60202E8
:1003800030B58C180278401C13071B0F01D103787D
:10039000401C120906D10278401C03E005780D705C
:1003A000401C491C5B1EF9D101E00B70491C521E18
:1003B000FBD1A142E6D3002030BD7047704700005A
:1003C000F0B581B001220092D303494A012918DB1C
:1003D0004118002503E0ADB2401C884212D2009CB7
:1003E00026020778BE1904E03D4674001E422646E8
:1003F000F1D16F003406E40FE7191D42F4D05740E5
:10040000F2E7002568001D4230D14100184231D189
:100410004800194232D14100184233D148001942F4
:1004200034D14100184235D14C00194236D1600018
:100430001C4237D10104C90B184238D14800194277
:1004400039D1410018423AD1480019423BD141000C
:1004500018423CD1480019423DD1410018423ED1DA
:10046000480019423FD180B201B0F0BD5040410078
:100470001842CDD0514048001942CCD050404100E4
:100480001842CBD0514048001942CAD050404100D8
:100490001842C9D051404C001942C8D054406000A5
:1004A0001C42C7D050400104C90B1842C6D051406D
:1004B00048001942C5D0504041001842C4D05140B4
:1004C00048001942C3D0504041001842C2D05140A8
:1004D00048001942C1D0504041001842C0D051409C
:1004E00048001942BFD0504080B201B0F0BDC046B4
:1004F00021100000B0B582B0194C2068056801A930
:100500000020087007E090470198401C01A908707E
:10051000C0B2082822D2012211048140294209D008
:100520002268516080002018826A002AECD001A85D
:100530000121E8E7130283402B4201D0022104E0AD
:1005400082402A42E0D00321134622685360800093
:1005500020188268002AD7D001A8D4E702B0B0BD25
:1005600010EC0202FEE7000010B509480168CA69F4
:1005700020231343CB610269032A08D1012293058A
:100580000C689C430C605102C26E0A43C26610BDE7
:1005900078EC0202F0B581B05C4C2068856BE8070E
:1005A00007D0E168002904D0002088472068012195
:1005B0008163A80707D52169002904D00120884755
:1005C000206802218163680707D56169002904D08A
:1005D00002208847206804218163280707D5A16984
:1005E000002904D003208847206808218163E80699
:1005F00007D5E169002904D004208847206810212C
:100600008163A80607D5216A002904D00520884700
:10061000206820218163680607D5616A002904D01B
:1006200006208847206840218163280607D5A16AF3
:10063000002904D007208847206880218163012693
:10064000E80507D5E16A002904D037020820884769
:1006500020688763A80507D5216B002904D077029D
:100660000920884720688763680507D5616B0029E2
:1006700004D0B7020A20884720688763280507D579
:10068000A16B002904D0F7020B20884720688763FC
:10069000E80407D5E16B002904D037030C20884714
:1006A00020688763A80407D5216C002904D077034C
:1006B0000D20884720688763680407D5616C00298E
:1006C00004D0B7030E20884720688763280407D525
:1006D000A16C002904D0F7030F20884720688763A6
:1006E000E80307D5E16C002904D0370410208847BF
:1006F00020688763A80307D5216D002904D07504FD
:10070000112088472068856301B0F0BDF4EC020237
:1007100010B5012044061920020306492046FFF7C0
:100720000BFE206880F3088860680019804700206D
:1007300010BDC04600A00004F0B585B00391074687
:1007400004906B4E08463146FFF7E0FD0446302525
:1007500028433870601E2746874166430398801BF4
:100760000390644E3146FFF7D1FD014602952943BF
:100770003D46049AD1552746074346430398801BBC
:100780005D4E01903146FFF7C1FD002C04D00222DE
:10079000002F049904D105E00122002F049901D013
:1007A000049989180246029B1A430A70002F00D050
:1007B0006D1CC4B203952C43049F00D04F1C4643CC
:1007C0000198851B4D4E28463146FFF79FFD014697
:1007D00030313970002C01D1039901E00399491C93
:1007E000C4B203910C43049A00D07A1C4643AD1B5B
:1007F000434E284631461746FFF788FD0146029AC8
:1008000011433A463970002C01D1039901E0039954
:10081000491CC4B203910C43049F00D0571C4643AB
:10082000AD1B384E28463146FFF770FD0146029A4F
:1008300011433970002C01D1039901E00399491C3F
:10084000C4B203910C43049900D0791C4643A81B01
:1008500080B20D467D21C900FFF758FD0A460146CA
:10086000303129702946002C05D1039F84B23C43C6
:10087000049D06D106E0039F7F1C84B23C43049D87
:1008800000D04D1C6426019210463146FFF73EFD14
:100890000146029A11432970002C00D07F1C039757
:1008A0000743049C019900D06C1C4643881BC5B2C9
:1008B0000A212846FFF72AFD029A10432070601C87
:1008C0000A2D0BD2002F0CD1039ABA4200D004900B
:1008D000029801430498017005B0F0BD0490002F08
:1008E000F2D00022D743039ABA42F1D0EFE7C046D4
:1008F00000CA9A3B00E1F5058096980040420F003F
:10090000A086010010270000F0B589B00446E02061
:10091000085C227842402270637804910846E030F7
:1009200042785A406270A17882784A40A270E17899
:10093000C2784A40E270217902794A4022714179B5
:1009400062794A4062718179A2794A40A271C17983
:10095000E2794A40E271017A227A4A402272417A6F
:10096000627A4A406272817AA27A4A40A272C17A5D
:10097000E27A4A40E272017B227B4A402273417B49
:10098000627B4A406273817BA27B4A40A273C17B37
:10099000E77B4F40E77320460C3003902046083039
:1009A0000290201D01900D200790D0200890627BBE
:1009B000617A6173637960780690607163726270C6
:1009C000A578A37AA370A572A579A67BA671A57355
:1009D000E678E0790590E070E07AE673E772E0711E
:1009E000049F0898395C2678664DAE5D4E402670AF
:1009F000AA5C3818467856406670EA5C83785340A3
:100A0000A37005996A5CC3785340E3702279AA5CAD
:100A10000379534023710699695C42794A406271B7
:100A2000A179695C82794A40A271E179695CC279F5
:100A30004A40E271217A695C027A4A402272617A04
:100A4000695C427A4A406272A17A695C827A4A4061
:100A5000A272E17A695CC27A4A40E272217B695CE7
:100A6000027B4A402273617B695C427B4A4062732D
:100A7000A17B695C827B4A40A273E17B695CC07B9D
:100A80004840E073204600F07FF8019800F07CF8C1
:100A9000029800F079F8039800F076F80799491E5B
:100AA000080605D00791089810380890E77B7EE784
:100AB000617B607A607362796078089060716272BD
:100AC0006170A378A27AA270A372A379A57BA571A5
:100AD000A373E578E079E070E67AE671E67BE5738A
:100AE000E6722578274B5D5D049F3E786E40267048
:100AF000595C7D784D406570995CBA784A40A27027
:100B0000195CFA784A40E2702179595C3A794A4096
:100B100022710898185C797941406171A079185C5C
:100B2000B9794140A171E079185CF9794140E171EE
:100B3000207A185C397A41402172607A185C797A9F
:100B400041406172A07A185CB97A4140A172E07AA2
:100B5000185CF97A4140E172207B185C397B414096
:100B60002173607B185C797B41406173A07B185CCA
:100B7000B97B4140A173E07B185CF97B4140E17394
:100B800009B0F0BD84F00202F0B58AB00746012139
:100B900041560891CA091B2632404800424005923E
:100BA00051004AB2D209324040B2C00930404840F8
:100BB000049041005140022038560990C309334047
:100BC0004000434007935A0053B2DB09334040B220
:100BD000C009304050400390400058404840032135
:100BE000795602910197CD09354049004D406A0080
:100BF00053B2DC09344049B2CB0933405340590069
:100C000061404140387844B20694600042B2D20953
:100C10003240E409344044406000424057000097AD
:100C200040B2C0093040009E7040484006460999D5
:100C30004E400699089F79404E406E406640049FA2
:100C40007B405E40019FFE70029E70404140079EC7
:100C500071406940039D6A4051403D46B97001466C
:100C6000099E7140069E7140059E7140079F794024
:100C7000594069700899484009994840704060405F
:100C8000504028700AB0F0BDF0B58AB00346FC2091
:100C90000790D877F92005909877BA200490587774
:100CA00021241C774A20D876A32098765B2058769A
:100CB000202018760025DD750820987507205875C6
:100CC000932018751926DE743320987405275F74F5
:100CD000132119742320D8730120987352225A7358
:100CE00030221A73D872CA229A72DE225A721822DD
:100CF0001A72DD7199711221597189211971DE7091
:100D0000042199705F7006931C70089009A80499DB
:100D1000417004700799C170059981701B20019082
:100D2000C043059008A8407800901C213BE009AA28
:100D300010782D498968085C0290D078085C03908F
:100D400050780D5C90780F5C00984740577008A869
:100D5000017849B204914D401570837803994B4056
:100D60009370C178029C6140D170049AD209019CB1
:100D70002240049C640054400470059C305D68402F
:100D800009AA10703071301944787C40547085780D
:100D90005D409570C0784840D0707471B571F07145
:100DA0000799EC291ED206984618091D1F200840F5
:100DB0000791BCD010280FD109A801780A4A92687F
:100DC000555C05704178575C47708178535C83703F
:100DD000C178515CC170D0E709A8C17883784778A1
:100DE0000578CAE70AB0F0BDE8ED0202F0B581B0BF
:100DF00000F0A8F800280BD0164801F0D4F8BFF393
:100E00004F8F154815490160BFF34F8F00BFFDE7B5
:100E10006C461348208001273A030025114E2846CE
:100E2000314601F067FC103602232846314622463F
:100E300002F0ECF97C06192002030B492046FFF76B
:100E40007BFA206880F3088860680019804701B049
:100E5000F0BDC046102700000CED00E00400FA05CC
:100E6000FFFF000000D0020400A000040648016853
:100E7000032291430160016801220A43026000F0ED
:100E800077FB02F093FFC0462800004080B50B4975
:100E90000868002800D480BD094802680423032A9A
:100EA00001D01A4300E01A460A6006490A68002A7F
:100EB000F1D041680020904780BDC0462C10014011
:100EC00000EC020250F6020280B500F00FF800209C
:100ED00080BD0000524909684A69D20501D400204A
:100EE00070474968017001207047C04680B582B0E4
:100EF00001A908704A480068416A0029FCD101A98B
:100F000001220020034603F0FDF902B080BDC04677
:100F1000B0B582B004460078002811D0404D01A938
:100F200008702868416A0029FCD101A9012200202B
:100F3000034603F0E7F9611C607800280C46EED107
:100F400002B0B0BD70B584B001A80026068102963B
:100F500001963320FFF7B8FF154800F04DFB04461B
:100F6000012819DB134800F041F8134800F03EF85F
:100F700001AD28462146FFF7DFFB10A000F036F850
:100F8000284600F033F810A000F030F811A000F06F
:100F90002DF8F0B204B070BD0220C043844203D3E8
:100FA0006642F0B204B070BD0426F0B204B070BD69
:100FB0006CF60202ACE5020284EE02020A0D205336
:100FC000697A653A200000002042797465730D0A41
:100FD000000000002D2D2D2D2D2D2D2D2D2D2D2DF5
:100FE0002D2D2D2D2D2D2D0A00000000B0B582B025
:100FF00004460078002811D0094D01A9087028681E
:10100000416A0029FCD101A901200023024603F016
:1010100079F9611C607800280C46EED102B0B0BDB1
:1010200048ED0202F0B5024603781C464B3C002016
:10103000222C16D87C4424796400A7441128112856
:101040002828282828282828282828282828282820
:101050002828282828282828282828281128110066
:10106000F0BD002B38D0302B11D1547820252543EA
:10107000782D10D19478002CF2D05623DB432546EE
:10108000413D062D00D356E01D4620355FE01C464D
:10109000303C092CE4D8303B55782C464B3C222C74
:1010A0001ED8C0467C4424796400A744111B401B11
:1010B0001B1B1B1B1B1B1B1B1B1B1B1B1B1B1B1B80
:1010C0001B1B1B1B1B1B1B1B1B1B1B1B111B400070
:1010D000980208600120F0BD03460B600120F0BDBE
:1010E000002DFAD02C46303C092CB9D80A24634391
:1010F0005B19303B95782E464B3E222E00D980E07E
:101100007E4436797600B744117F127F7F7F7F7FE0
:101110007F7F7F7F7F7F7F7F7F7F7F7F7F7F7F7FDF
:101120007F7F7F7F7F7F7F7F117F1200D0E7180551
:1011300008600120F0BD2546613D062D1D4606D301
:101140002546303D092D00D98AE71D4627352C1943
:10115000D578002D00D1D8E02E46413E062E02D291
:101160001E4620360BE02E46613E062E1E4606D356
:101170002E46303E092E00D972E71E4627367519D5
:1011800024012C191579002D00D1BEE02E46413ED8
:10119000062E02D21E4620360BE02E46613E062E5B
:1011A0001E4606D32E46303E092E00D958E71E466D
:1011B0002736751924012C195579002D00D1A4E08A
:1011C0002E46413E062E02D21E4620360BE02E460B
:1011D000613E062E1E4606D32E46303E092E00D90D
:1011E0003EE71E462736751924012C199579002DE6
:1011F00000D18AE02E46413E062E2BD21E462036D6
:1012000034E0002D00D168E72E46303E092E00D98B
:1012100026E763435B19303BD5782E464B3E222EA2
:1012200000D975E07E4436797600B74412741174A3
:10123000747474747474747474747474747474746E
:101240007474747474747474747474741274110097
:101250006DE73DE72E46613E062E1E4606D32E461E
:10126000303E092E00D9FBE61E46273675192401AB
:101270002C19D579002D48D02E46413E062E02D29B
:101280001E4620360BE02E46613E062E1E4606D335
:101290002E46303E092E00D9E2E61E462736751945
:1012A00024012C19157A002D2FD02E46413E062EF2
:1012B00002D21E4620360BE02E46613E062E1E460A
:1012C00006D32E46303E092E00D9C9E61E462736E3
:1012D000751924012C19557A002D16D02E46413E41
:1012E000062E01D2203309E02E46613E062E05D39C
:1012F0002E46303E092E00D9B2E62733927A002AD4
:1013000000D0ADE65819220184180C600120F0BD10
:10131000002D00D1E1E62E46303E092E00D99FE691
:1013200063435B19303B15792E464B3E222E17D86E
:101330007E4436797600B744121611161616161624
:10134000161616161616161616161616161616163D
:10135000161616161616161612161100E7E6B7E63A
:10136000002D00D1B9E62E46303E092E00D977E691
:1013700063435B19303B55792E464B3E222E17D8DE
:101380007E4436797600B7441216111616161616D4
:1013900016161616161616161616161616161616ED
:1013A000161616161616161612161100BFE68FE63A
:1013B000002D00D191E62E46303E092E00D94FE691
:1013C00063435B19303B95792E464B3E222E17D84E
:1013D0007E4436797600B744121611161616161684
:1013E000161616161616161616161616161616169D
:1013F00016161616161616161216110097E667E63A
:10140000002D00D169E62E46303E092E00D927E690
:1014100063435B19303BD5792E464B3E222E17D8BD
:101420007E4436797600B744121611161616161633
:10143000161616161616161616161616161616164C
:101440001616161616161616121611006FE63FE639
:10145000002D00D141E62E46303E092E00D9FFE591
:1014600063435B19303B157A2E464B3E222E17D82C
:101470007E4436797600B7441216111616161616E3
:1014800016161616161616161616161616161616FC
:1014900016161616161616161216110047E617E639
:1014A000002D00D119E62E46303E092E00D9D7E591
:1014B00063435B19303B557A2E464B3E222E17D89C
:1014C0007E4436797600B744121611161616161693
:1014D00016161616161616161616161616161616AC
:1014E0001616161616161616121611001FE6EFE53A
:1014F000002D00D1F1E52E46303E092E01D9FFF72F
:10150000AFFD5C436319303B927A14464B3C222C6E
:101510001BD8C0467C4424796400A74414121112DD
:10152000121212121212121212121212121212129B
:10153000121212121212121212121212141211009C
:10154000F5E5FFF78DFDFFF7C3FD002A01D0FFF79A
:1015500087FDFFF7C2FD000080B504480168491C03
:1015600001600069002800D0804780BD54F6020267
:1015700001480249016070470CEC02020026B803E2
:1015800080B582B00E4908680022C2600192CA6824
:10159000002A02D0016801A8904702B080BDC04671
:1015A00080B582B0064908690022C260012201921A
:1015B000CA69002A02D0016801A8904702B080BD24
:1015C00058EC020280B5002002F0CAFC80BD80B554
:1015D000012002F0C5FC80BD80B582B000200190E2
:1015E0000448C268002A02D001A80021904702B036
:1015F00080BDC046D8ED0202F0B583B0044600F0CD
:1016000091F9C14D00210220A8806980BF48E8609F
:1016100029616961A96101910294E96129626C62A1
:10162000A962BB4C641C00D3BAE02846FFF752FC09
:101630000128F7D12878411E172900D9ABE0802274
:101640000092C0467944097949008F440E0BA94A9B
:10165000A9A9A9A9A9A9A9A9A9A9A9A9A9A9A9A9FA
:10166000A9A9A9980121890200910121E980A94B2A
:1016700018700524009804435E18A54F7F1C00D302
:101680008EE03046FFF726FC0128F7D1E888401CA1
:10169000E88081B28C429F4BEED89878FF2242407E
:1016A0005978914200D0FAE06888884203D02978BE
:1016B000012900D0F3E0401C6880964CE01C009E9D
:1016C0003146FEF77DFE04213143615C0322324343
:1016D000A25C12025118814200D0E0E0009AAA6296
:1016E00000E0AA6A00266E61002A029C00D1C2E0D6
:1016F000501C00D1EEE087484178E869C3B29942B6
:101700005FD100285FD0686A8249C91CFEF714FEC9
:101710006C63AE63AB6A012B0DDB20462946443176
:1017200000F062F9686B10306863A96B1031A9632F
:10173000AB6A9942F2DB6888800277494018EC6313
:101740002864E96800273846224601F05FFD00283A
:1017500000D0B0E0296CE868884203D0AA689142C2
:1017600000D8A8E0A96A0818E8600620FFF7BEFBC9
:101770006A480760A888401CA88001996EE0644C04
:10178000641C0DD22846FFF7A5FB0128F8D1287864
:10179000182805D19AE0412800D180E061287ED048
:1017A0006869A969012901DB401C6861029C06285F
:1017B0006BDA4320FFF79AFB0199286A002856D17B
:1017C0002EE71520F6E7534BD878002800D187E0A4
:1017D000D81CEE622863524C9919C878A055701C29
:1017E0000A1DE8622A630979002902D0FF2E064605
:1017F000F2D3002121541818021DE9622A630279EC
:10180000202A0A460FD00023EA18C4182679542744
:10181000D6555A1C661DEA622E636479202C02D0CC
:101820000E2B1346F0D3501CE862284654308154E6
:1018300029460831FFF7F6FB19200203501CA9685E
:10184000814256DC0020314900F054FF0620FFF7AA
:101850004DFB4320FFF74AFB0199029C0120A86140
:10186000E869401CE861286A002800D1D8E62869A8
:1018700000283BD1D1E60620FFF738FB0120286283
:1018800001992869002831D1C7E618252846FFF7B5
:101890002DFB2846FFF72AFB019803B0F0BD182462
:1018A0002046FFF723FB2046FFF720FB0020C04324
:1018B000801E03B0F0BD18242046FFF717FB20461A
:1018C000FFF714FBF843401E03B0F0BD01986861B8
:1018D000C043A8620620FFF709FB019803B0F0BDE2
:1018E0000620FFF703FB012028612862A86803B0E7
:1018F000F0BD18242046FFF7F9FA2046FFF7F6FA64
:101900000020C04303B0F0BDFCED020200A00004C3
:10191000FFFFEFFF48F20202009C000468EE0202A3
:1019200084EE0202F0B581B07B4C2D4F2D4EC0C429
:1019300001220021083CD3B2F954CBB2F254530037
:1019400053401206D5171B222A405A40D3B2491CD5
:10195000012BF0D13278FF2032546E49A16063230D
:101960000B700026BD196D7845401E494D5D394606
:10197000EF096A00D2192F46574052006C06E40F57
:10198000121957405200AC06E40F1219574052008A
:10199000EC06E40F12197A400F465A405D498C1943
:1019A0006270761CFF2EDDD15B4C0E48E060FFF7C5
:1019B0006BF92761A06800210A4605E0BB54521C60
:1019C00001231B029A4209D00B46DDB2445DA242BC
:1019D000F4D06B1CDCB29C42F7D0F0E701B0F0BD54
:1019E00084F0020284EF0202F0B585B00C46054691
:1019F000FFF798FF2878474E307068780490A878F1
:101A00000390E8780290287901906F79AA79E979B2
:101A1000287A6B7A73723072F171B27177710198B2
:101A200030710298F0700398B07004987070A87AC2
:101A3000B072E87AF072287B3073687B7073A87B91
:101A4000B073E87BF0733448C1682846FEF75CFF4A
:101A50002078297841402970687861784140697020
:101A6000A878A1784140A970E878E1784140E97010
:101A700028792179414029716079697941406971FA
:101A8000A079A9794140A971E079E9794140E971EA
:101A9000207A297A41402972607A697A41406972D4
:101AA000A07AA97A4140A972E07AE97A4140E972C4
:101AB000207B297B41402973607B697B41406973AE
:101AC000A07BA97B4140A973E07BE97B4140E9739E
:101AD0003078207070786070B078A070F078E07026
:101AE0003079207170796071B079A071F079E0710E
:101AF000307A2072707A6072B07AA072F07AE072F6
:101B0000307B2073707B6073B07BA073F07BE073DD
:101B100005B0F0BD6CFA0202E8ED020270B517489C
:101B20004C210160FF240234204600F0F3F83220FB
:101B300000F039FA00F0DCF80125284600F0E2F860
:101B4000284600F033F800F0CDF80D4800F0E2F838
:101B500000263046314600F0EDF92846314600F0C7
:101B6000E9F9304600F0D6F8022000F0D3F8473407
:101B7000204602F01FF902F039F970BD480000401C
:101B800001020000704710B505200424214601F031
:101B900025FF0620214601F021FF0A20214601F001
:101BA0001DFF0920214601F019FF10BD02490A68F6
:101BB00002408242FBD1704704600040B0B53C480F
:101BC00001688A073B4C07D501797F221140E36900
:101BD00093435918E1610168890407D55E21405C8F
:101BE0007F210840226A8A4310182062172000F0E3
:101BF00011F93148016802220A4301218A43026037
:101C00002E482F4901602F480021C17181791F257D
:101C100029408171817A427C837C1B029A18C37CA3
:101C20001B04D218037D1B06D218274B9A4218D1E9
:101C3000427B837B1B029A18C37B1B04D218037C54
:101C40001B06D218214B9A420BD1C27A037B491E44
:101C5000122906D8190289181D4A914201D1202162
:101C600001720178CA0602D1102211430170206866
:101C700020218843206026481649016041680029D8
:101C8000FCD502F07FF80A21C841032800D8FEE7FE
:101C90001148C1680F229143C16001680F4A0A4090
:101CA0000260192000010E4948600D60B0BDC046B9
:101CB00084F102022C000040040200400C060040A7
:101CC000AF6B100A6B0001404D383650312E323662
:101CD00007340000FE1C0080C8600040FEFFC3FF08
:101CE0000C04004080B5172000F08CF8002080BD67
:101CF00010B51724204600F08DF8204602F048F871
:101D0000002010BD0121C90701430148016070474F
:101D10000060004010B5C1B2000AC2B202290CD066
:101D2000012913D0002930D1911E7F4802291BD2EE
:101D30000121032A2AD0490429E07B484168002A6E
:101D40001FD00246203A1143416010BD7648016819
:101D5000D31E022B10D3012A29D0002A41D10122FF
:101D600092079143016010BD002A16D10121490755
:101D700002688A43026010BD0123042A1FD05A045E
:101D80001EE0012292079143416010BD0904194AE7
:101D90007F32C36A13405918C16217498A69920792
:101DA000FCD50121490702680A43026010BD0522E3
:101DB000120791430246203A0A43026010BD1A04FA
:101DC000836A0C4C1C40A21882620B4A131F002429
:101DD0001C600A4B0A4C1C600D235B0214681C43F8
:101DE0001460054A93695B06FCD50522120711436E
:101DF000016010BD80FFFCFF1402004004010040A0
:101E0000FF0F000001218140474802688A430260B9
:101E10007047C04601218140434802680A4302607E
:101E20007047C04610B5052811D8C04678440079DF
:101E300040008744020E192434393B490A68086877
:101E4000C0003CD53A4820390A425DD03BE0002032
:101E500010BD35490A680868C00035D534480B46BE
:101E6000203B1A4237D134E02F490A680868C00085
:101E700036D52F480B46203B1A424CD135E02A4933
:101E80004C680120C0030A680B46203B1C421AD054
:101E90000C68E4003BD5264C1A423CD03AE022487C
:101EA00000680120C00310BD1F490A680868C0000F
:101EB0001ED51F480B46203B1A4220D11DE01B486F
:101EC00020390A4220D010BD18480B46203B1A4248
:101ED00001D10120C00349688900890FC84010BDA5
:101EE00012480B46203B1A4215D10120C00312E0D4
:101EF0000E480B46203B1A4201D10120C00349681D
:101F00000903890FC84010BD0120C00310BD074C54
:101F10001A4200D020464A689200920FD040496889
:101F20000901890FC84010BD20000040006CDC0290
:101F30000026B80304282CD8164AC04678440079F5
:101F400040008744020A121A210003200007136888
:101F500083438807800818181AE003208006136856
:101F6000834388070009181812E0032080041368CF
:101F700083438807000B18180AE0FF20000213684B
:101F800083430802181803E01068FF2398434018A1
:101F9000106070472400004080B57D21C90048438F
:101FA00000F001F880BD00280AD030B407252C02CB
:101FB000CD256419604340091238001FFDD830BC9C
:101FC00070470000F0B581B005460120072D66D8A6
:101FD0000C46002963D0464F38680169C90736D1DD
:101FE00005263046FFF716FF304601F0D1FE03CF3D
:101FF0000369012213430361002918D403200B460F
:10200000834370481E588807C00EFF278740BE4391
:102010004027874037436B481F501F2008408240AD
:102020006948026069480260314800680FE08A0729
:10203000D20EFF2696400F230B40083B03218B4313
:102040005F495F58B743402696403E435E50690162
:102050004018012109024218E369DB069B0CA569BF
:10206000ED00EDB2EB18536062685207520B236823
:102070005B075B099A18A3685B079B0CD218E3689F
:102080005B075B0DD21823695B01DBB2D218636971
:102090009B07DB0ED218802313434350002001B06E
:1020A000F0BDC046F0B581B005460835104C266835
:1020B000F668EE40F50702D0022001B0F0BD069DA3
:1020C0008600A619B56040012468201800930123FA
:1020D0001D02461977680724A7437760F1603261D3
:1020E0000099B160415919434151002001B0F0BD40
:1020F00010EC020200013B49085840687047C04696
:10210000F0B581B005460120012D45D80C460029C7
:1021100042D0002D03D0012D04D10F2000E00E206D
:10212000FFF778FE29012F4843580020D860276820
:102130006568A668F607B60FAD072D0FAE192569BD
:10214000EA07920EB618022F04D0012F03D1012204
:10215000164300E040369E60E2681A60214A51183A
:102160008D606269CA604968002917D403220B4652
:102170009343144A9C588D07ED0EFF26AE40B4439E
:102180008026AE4026439E501F220A4001219140E6
:102190000D4A11600D4A116001B0F0BD8A07D20EE0
:1021A000FF2494400F230B40083B03218B43044939
:1021B0005D58A543802494402C435C5001B0F0BD91
:1021C0001CED00E000E400E080E200E000E100E05F
:1021D0000001044A10580160816880220A4382602D
:1021E0007047C04658EC0202F0B583B0019101235C
:1021F000EFF31081194002D1EFF3108272B67C2404
:1022000002904443C94807193A46103200923A698D
:102210000025062A0CD81E469640F206520F06D11B
:102220006122164271D01D46002903D003E0022529
:10223000002900D162B6002D02D0284603B0F0BDBF
:1022400000591021C1613E46143601F0C9FD054612
:102250003868C069C00605D501F0C2FD401B318851
:102260008842F5D90621029D284600F049FF386AC8
:1022700001994143B8690918386881601721795676
:102280003C461734002909D5C16920220A43C2619E
:102290000121F966890502680A4302600521284682
:1022A00000F02EFF207840B200250028C5D41A483F
:1022B00000687D24E100FEF729F86101414302989E
:1022C00000F0D0FD01F08CFD04463868C069C007FD
:1022D00005D001F085FD001B31888842F5D901F059
:1022E0007FFD04463868C169890706D501F078FD8D
:1022F000001B31888842F5D938680121009A1160A5
:1023000042498161284603B0F0BD0322009B1A6058
:1023100000298FD08FE7C04668F60202F0B583B07F
:1023200002907C214143EF4A5418E56EEAB2511EF7
:1023300002291FD229040126090E18D00196009205
:10234000022100F0DDFE2746143701F049FD064664
:102350002068C169890606D401F042FD801B3988D6
:102360008842F5D92068007DC007019E08D030461C
:1023700003B0F0BD032A36D100922804000E36D0F7
:1023800020466C302D0C0021019101602746143746
:1023900001F026FD06462068C069C00705D001F09F
:1023A0001FFD801B39888842F5D901F019FD0646CA
:1023B0002068C169890706D501F012FD801B3988A4
:1023C0008842F5D9206811498161E9B201200029CC
:1023D00011D003290099019E00D006202061226FB0
:1023E000002A0ED1C3E70026304603B0F0BD012617
:1023F000304603B0F0BD0099019E2061226F002A93
:10240000B5D002A89047304603B0F0BD000093EB72
:10241000F0B581B00C460078B24EF16881422CD103
:10242000032C54D1706EB16E884261D9002406210C
:10243000204600F065FE3068F16D8160204621463F
:1024400000F05EFE354660352CCDF0683168B48C06
:10245000374F00975B1BA34200D81C46A3081431DA
:10246000FFF720FEB06E0019B066306E00193066BE
:10247000F06D0019F06501B0F0BDB168814224D162
:10248000032C45D1F08CF16D0918F165316E0918F6
:102490003166B16E0818B066716E814238D9002479
:1024A0000621204600F02CFE3068F16D816001218C
:1024B000204600F025FE316EB068F38C32681C4C6B
:1024C000009414329B08FFF7EDFD01B0F0BD3068B9
:1024D0001021C16101F084FC05463068C069C00666
:1024E00016D501F07DFC401BB18A8842F5D90FE07A
:1024F00030681021C16101F073FC05463068C06985
:10250000C00605D501F06CFC401BB18A8842F5D9A4
:102510000120C107326813688B431360F16E2204F7
:102520000A4300021043F06601B0F0BD78EC0202ED
:10253000D9C10202F0B581B00078C14DAA688242CB
:1025400050D101263002032942D16A6DAA66AB6DD3
:10255000AC6AA418EB652C66AB6C5B1CAB646B6E51
:10256000934235D95E30FFF71EFD686CA96C0229D5
:102570003AD3814238D1E88C696D0818686500202B
:10258000062100F0BDFD2868E96D81602F6D01F026
:1025900027FC04462868C069C00705D001F020FC6C
:1025A000001BA98A8842F5D901F01AFC04462A6862
:1025B000D069800706D501F013FC001BA98A884268
:1025C000F5D92A687420285C012841D0F10440E044
:1025D000F2072B681C6894431C60EA6E09041143DF
:1025E0000143E96601B0F0BD0229FBD38142F9D273
:1025F000E88C696D09186965A96D0818A86500203F
:10260000062100F07DFD2868E96D8160EF8C01F006
:10261000E7FB04462868C069C00705D001F0E0FB6D
:10262000001BA98A8842F5D901F0DAFB04462A6822
:10263000D069800706D501F0D3FB001BA98A884228
:10264000F5D92A687420285C012822D0F10421E001
:102650003105254B3B405918012802D0192040066E
:1026600001E00720C0060818204940185060002FDC
:102670000DD001F0B5FB04462A68D069800706D466
:1026800001F0AEFB001BA98A8842F5D92A682B6DA0
:102690001FE03105144B3B40C918012802D0192016
:1026A000400601E00720C006081810494018506095
:1026B000002F0DD001F094FB04462A68D0698007F2
:1026C00006D401F08DFB001BA98A8842F5D92A683F
:1026D000EB8C296EA868064C00941432FFF7E2FCDC
:1026E00001B0F0BD78EC0202FF3F000000808000E6
:1026F000FDC20202F0B587B004460126880E14D050
:102700001546002A11D00F468120C004401B884284
:102710000BD37C206043EB4908180590818C384628
:102720000691FDF7F3FD002902D0304607B0F0BD59
:1027300028460699FDF7EAFD0029F6D1059880693B
:102740003E1A30460699FDF7E1FD074603967019DB
:102750000190069E3146FDF7D9FD0546C01B049049
:102760000598006A02903146FDF7D0FD0499814238
:102770000FD20026BD42D8D92046394600F0D6FAFD
:102780002046FFF7CBFD0028FAD17F1CAF42F3D3E0
:10279000CBE700900398029D2946FDF7B7FD06465A
:1027A000284670430399081A019800D0761C2946E0
:1027B000009D7543FDF7AAFD0590029941430198DC
:1027C000401A03900699FDF7A1FD0490AF420BD289
:1027D0002046394600F0AAFA2046FFF79FFD002860
:1027E000FAD17F1CAF42F3D305988642069D009F25
:1027F0000CD220463146FFF7F7FC2046FFF78EFD4E
:102800000028FAD1761C05988642F2D30398A84294
:1028100003D20026304607B0F0BD05984743002597
:10282000E919204600F082FA2046FFF777FD0028DC
:10283000FAD16D1C002604988542F1D375E7C04695
:1028400078EC0202F0B585B0002803D001242046C0
:1028500005B0F0BD78209B4F0490385C002803D071
:102860000024204605B0F0BD002905D038461430BC
:102870000CC90CC01CC91CC00020F86615242046D9
:10288000FFF7C8FA204601F083FA38681021C161C9
:1028900001F0A6FA04463868C169C90607D501F0F7
:1028A0009FFA001BB98A8842F5D9386800E0B98AD6
:1028B000BA7D1207120B5218F97DCB07DB08D2182C
:1028C0008B07DB0F5B05D218CB06DB0FDB05D218BD
:1028D0004B07DB0FDB06D2188B06DB0F5B07D2182A
:1028E0000907C90F89071143016000240A21204606
:1028F00000F006FC3220FFF756FB0821204600F0CE
:10290000FFFB01F06DFA05463868C169890606D4F7
:1029100001F066FA401BB98A8842F5D93868017D12
:102920000A46C23A534253417426BB55027D007D8C
:10293000C22919D1F87D039000250621284600F010
:10294000DFFB0721284600F0DBFB012103988143D0
:10295000B85D012847D13868890101750575752171
:10296000795C012938D048E003960020032100F06B
:10297000C7FB01F035FA05463868C169890606D4F7
:1029800001F02EFA401BB98A8842F5D93868007DDB
:1029900045080122F87D014629431540C90701D0A9
:1029A000284035D0002606213046029200F0A8FBD0
:1029B00007210196304600F0A3FB0298454003989A
:1029C000385C012813D13868A90101750199017596
:1029D0007521795C012910D114307621795C4A4245
:1029E0004A41510008E038680575490003E038683D
:1029F00001990175690014300170334800687D2128
:102A0000C900FDF783FC28214143002000F02AFA89
:102A10007720385C012803D102200021FFF78AFAD1
:102A200001F0DEF905463868C069C00705D001F03D
:102A3000D7F9401BB98A8842F5D901F0D1F905468A
:102A40003868C169890706D501F0CAF9401BB98AFF
:102A50008842F5D93868B449816117203856002872
:102A600029D57868002816D4032102468A431849DC
:102A700053588507ED0EFF26AE40B3438026AE4087
:102A80001E4356501F210140012088401149086013
:102A9000114908600FE08107C90EFF238B400F2208
:102AA0000240083A03208243084815589D4380237A
:102AB0008B402B43135001200499785438612046F1
:102AC00005B0F0BD78EC020268F602021CED00E0F1
:102AD00000E400E080E200E000E100E0F0B593B047
:102AE00001258C0E32D0002B30D009928122D204E5
:102AF0000693D21A08918A4228D30123EFF310815A
:102B0000194002D1EFF3108272B67C220A90424340
:102B1000EB4887183C46103405943E690025062E84
:102B20000ED81C46B440E606760F08D16126344222
:102B300000D1C9E01D460A9C002904D004E002250A
:102B40000A9C002900D162B6002D02D0284613B09D
:102B5000F0BD805810210491C1613E46143601F049
:102B60003FF905463868C069C00605D501F038F957
:102B7000401B31888842F5D9F87D400665D402961D
:102B8000BD8C069C20462946FDF7C0FB07902946D0
:102B90004143601A03903E462436A54200D89BE08C
:102BA000039800281CD006210A9C204600F0A8FAB1
:102BB000308807994843089940183968886000258B
:102BC0002046039C294600F09BFA079B099A30880F
:102BD000584340193968097D11546D1CA542F6D33C
:102BE00038680499C16101F0FBF80446029D386819
:102BF000C069C00605D501F0F3F8001B298888429A
:102C0000F5D901F0EDF804463868C069C00705D071
:102C100001F0E6F8001B29888842F5D901F0E0F8B8
:102C200004463868C169890706D501F0D9F8001B48
:102C300029888842F5D938680121059A11608849A8
:102C400081610025284613B0F0BD03200025089EB1
:102C5000FE650999396606997966BD66F8660120B0
:102C6000C00739680A6802430A600621204600F05E
:102C700047FA386886602046294600F041FA28491C
:102C80000BAA0A9259C959C259C959C2BC8CF868D1
:102C90000A99FFF797F9F8683968224A0092069A6C
:102CA000944200D31446A3081431099AFFF7FAF9A5
:102CB000B86E0019B866386E00193866F86D0019DC
:102CC000F865284613B0F0BD0223059C23600A9CDA
:102CD000002900D137E737E7002404E0641C079897
:102CE000844200D35CE706210A9800F009FA308894
:102CF0006043089940183968886000250A98294679
:102D000000F0FEF930880028099AE7D060431018D7
:102D10003968097D41556D1C30888542F6D3DDE761
:102D200090E40202D9C10202000093EBF0B583B037
:102D300001910123EFF31081194002D1EFF31082CA
:102D400072B67C2402904443E84807193A46103290
:102D500000923A690025062A0CD81E469640F206D3
:102D6000520F06D16122164273D01D46002903D0AE
:102D700003E00225002900D162B6002D02D02846CA
:102D800003B0F0BD00591021C1613E46143601F078
:102D900027F805463868C069C00605D501F020F857
:102DA000401B31888842F5D90621029D284600F053
:102DB000A7F9B88C01994143B8690918386881604E
:102DC000172179563C461734002909D5C1692022BC
:102DD0000A43C2610121F966890502680A4302605B
:102DE0000421284600F08CF9207840B22C460025BA
:102DF0000028C4D4C04800687D21C900FDF786FAC8
:102E00004B21C9004143204600F02CF800F0E8FFB8
:102E100004463868C069C00705D000F0E1FF001B18
:102E200031888842F5D900F0DBFF04463868C16973
:102E3000890706D500F0D4FF001B31888842F5D9F8
:102E400038680121009A1160AC498161284603B0BD
:102E5000F0BD0322009B1A6000298DD08DE7C0468B
:102E6000000093EBF0B583B001917C2202904243C5
:102E7000E3498C182546143500F0B2FF06460221BE
:102E8000029800F03DF900F0ABFF07462068C169E9
:102E9000890606D400F0A4FFC01B29888842F5D912
:102EA0002068007DC00708D06420FFF77CF800F0A0
:102EB00097FF801B01998842E1D903B0F0BDC0465D
:102EC00078EC0202F0B595B00D460127890E16D0B8
:102ED000002B14D08121C904C91AA9420FD30B9722
:102EE000099308927C274743C549CE190A90F48C70
:102EF00028462146FDF70AFA002903D00B9F3846E1
:102F000015B0F0BD07970C9609982146FDF7FEF91C
:102F100000290B9FF3D10121EFF31080084002D16B
:102F2000EFF3108272B60C9A16461036136900271A
:102F3000062B0DD80A469A40D3065B0F04D16123B5
:102F40001A4203D00F4603E0022701E0042131605A
:102F5000002800D162B6002FD1D10C9C2246263227
:102F60000798A74908581021C16127461437204601
:102F700018300490A069281A0590069211880791CC
:102F8000FDF7C4F90B900998059908180799FDF702
:102F9000BDF9059000F024FF07902068C069C006C5
:102FA00006D500F01DFF0799401A39888842F4D9E8
:102FB000E07D40063ED4029703960B9D05998D4215
:102FC0000A9C6BD20026069F11E04B4800687D21C9
:102FD000C900FDF79BF9099941430A9C2046FFF778
:102FE00041FF761C0B9D6D1C05998D4256D2398888
:102FF000079106212046099100F082F838880B9548
:1030000068430499096840180C990968886001218F
:10301000204600F075F838880028D6D0079A724309
:10302000089989180C9A12680B781375491C401E70
:10303000FAD1CAE702200027E565089921660999B7
:103040006166A766E0660125E80721680A68024311
:103050000A6006210A9E304600F052F8E06D2168B1
:1030600088603046294600F04BF821480DA90A46F1
:1030700078C878C278C878C20C9CA068FEF7A2FF16
:10308000A068216E069A138822681A4C00941432A4
:103090009B08FFF707F8384615B0F0BD00F0A0FE1A
:1030A0000446029E0C980068C069C00705D000F075
:1030B00097FE001B31888842F4D900F091FE044647
:1030C000039D0C980068C169890707D500F088FE48
:1030D000001B31888842F4D90C98006801212960CE
:1030E000064981610027384615B0F0BD78EC020230
:1030F00070E40202D9C1020268F60202000093EBFA
:10310000F0B585B0049104467C2060433C490F181B
:103110003D46143500F064FE06463868C069C007B5
:1031200005D000F05DFE801B29888842F5D900F0AB
:1031300057FE06463868C069800705D500F050FE86
:10314000801B29888842F5D91421049B5943DC202F
:1031500060432C4A1018039002914018018A82683B
:10316000C47C7426BE5D012E0DD10191012B029904
:103170000CD0012B0DD07526BE5D012E0ED0019E08
:10318000072B0ED10EE00E4602990BE00222012B16
:10319000F1D138247526BE5D012EF0D10326072B10
:1031A00000D0019E184B334024069207D20A121910
:1031B000D218039B5958C907490C52184168CB07CC
:1031C0001B0CD218837C5B075B0BD218C0684007CE
:1031D000000A10183A685060002E0ED001290CD158
:1031E00000F0FEFD04463868C069800705D400F091
:1031F000F7FD001B29888842F5D905B0F0BDC0460F
:1032000078EC0202D0E40202FF3F0000F0B59DB06E
:103210000D460126890E2FD0002B2DD01192812131
:10322000C9041093C91AA94226D30121EFF31084CF
:103230000C4002D1EFF3108272B67C220F90424311
:10324000E74814928718384610303B690026062B51
:103250000DD80A469A40D3065B0F07D161231A4264
:1032600000D16FE30E46002C03D003E00226002CB1
:1032700000D162B6002E02D030461DB0F0BD0290E3
:10328000BD650021139179651098401E1290401978
:10329000B964B9690D916E1A1199B962FD6238630A
:1032A0007E63F98C0E913046FDF730F80446B86322
:1032B000129830180E9E3146FDF728F8109B011B1E
:1032C0004A1CF86339647A64139A0029194608D0B5
:1032D000704359190D9BC91A0A1A7443581B801957
:1032E0000119384648300E90384644300D90384623
:1032F00040300B90384626300590384658301390B1
:10330000384654301290F9643A651498B449085814
:103310001021C16138461430149038465030049062
:103320003D464C3500F05CFD04463868C069C00677
:1033300006D500F055FD001B149909888842F4D980
:10334000F87D40060C9500D574E201230E980360C9
:103350000D98016800290F9800D1CDE23A467432E9
:103360000A92DA0407921A05099219225206069265
:103370000722D206089216E09A4800687D21C9000B
:10338000FCF7C4FF109941430F9C2046FFF76AFDEC
:1033900020460C9D0E9A11684B1C13600D9909680C
:1033A0008B4200D9A8E20B9A1268012A55D0002A54
:1033B00000D0A8E02E6812990C6813990D680621B8
:1033C0001091FFF79DFE386885601198051900F08F
:1033D00007FD04463868C069C00706D000F000FD4C
:1033E000001B149909888842F4D900F0F9FC0446BE
:1033F0003868C169890707D500F0F2FC001B1499F1
:1034000009888842F4D938680A990A78012A089903
:1034100000D00699012A099A00D0079A3346724CC7
:10342000234013430B4371490B434360002EA3D049
:1034300000F0D6FC04463868C069800706D400F066
:10344000CFFC001B149909888842F4D93868297880
:1034500001756D1C761EFAD18EE7012B00D0C7E0F6
:103460002E6812990C6813990D6806211091FFF7C8
:1034700047FE386885601198051900F0B1FC0446D4
:103480003868C069C00706D000F0AAFC001B149978
:1034900009888842F4D900F0A3FC04463868C16961
:1034A000890707D500F09CFC001B14990988884205
:1034B000F4D938680A990A78012A089900D006993F
:1034C000012A099A00D0079A3346474C23401343F8
:1034D0000B4346490B434360002E69D000F080FC4B
:1034E00004463868C069800706D400F079FC001BE8
:1034F000149909888842F4D93868297801756D1CB7
:10350000761EFAD154E0012B00D0C9E02E68129942
:103510000C6813990D6806211091FFF7F1FD3868CA
:1035200085601198051900F05BFC04463868C06995
:10353000C00706D000F054FC001B1499098888428B
:10354000F4D900F04DFC04463868C169890707D5F5
:1035500000F046FC001B149909888842F4D93868A9
:103560000A990A78012A089900D00699012A099A2D
:1035700000D0079A33461C4C234013430B431B498E
:103580000B434360002E13D000F02AFC0446386839
:10359000C069800706D400F023FC001B1499098839
:1035A0008842F4D93868297801756D1C761EFAD1E5
:1035B0000C4800687D21C900FCF7A8FE1099414322
:1035C0000F9C2046FFF74EFC20460C9D2A68139B5B
:1035D000196889181960129B196889181960D9E649
:1035E00078EC020268F60202FF3F000000808000D3
:1035F0008B4200D0CEE604990E6812990C6813999C
:103600000D6806211091FFF77BFD386885601198E1
:10361000051900F0E5FB04463868C069C00706D00C
:1036200000F0DEFB001B149909888842F4D900F0F1
:10363000D7FB04463868C169890707D500F0D0FB7D
:10364000001B149909888842F4D938680A990A78C5
:10365000012A089900D00699012A099A00D0079AF0
:103660003346D44C234013430B43D3490B434360AD
:10367000002E00D180E600F0B3FB04463868C06934
:10368000800706D400F0ACFB001B1499098888421F
:10369000F4D93868297801756D1C761EFAD16BE66D
:1036A000129A1268119CA618139A15688B425FD162
:1036B00004990C6806210391FFF722FD38688560A4
:1036C00000F08EFB05463868C069C00706D000F0E0
:1036D00087FB401B149909888842F4D900F080FBCD
:1036E00010900C9D3868C169890708D500F078FBF7
:1036F0001099401A149909888842F3D938680A99B0
:103700000A78012A089900D006991091012A099A8D
:1037100000D0079A2346A7490B40134310990B4347
:10372000A5490B434360002C14D000F059FB1090C6
:103730003868C069800707D400F052FB1099401A1E
:10374000149909888842F3D9386831780175761C54
:10375000641EFAD19A4800687D21C900FCF7D6FDA5
:10376000039941430F9C2046FFF77CFB204611E65E
:1037700005990C8806210391FFF7C2FC3868856023
:1037800000F02EFB05463868C069C00706D000F07F
:1037900027FB401B149909888842F4D900F020FBCC
:1037A00010900C9D3868C169890708D500F018FB96
:1037B0001099401A149909888842F3D938680A99EF
:1037C0000A78012A089900D006991091012A099ACD
:1037D00000D0079A234677490B40134310990B43B7
:1037E00075490B434360002C14D000F0F9FA109097
:1037F0003868C069800707D400F0F2FA1099401ABF
:10380000149909888842F3D9386831780175761C93
:10381000641EFAD16A4800687D21C900FCF776FD74
:10382000039941430F9C2046FFF71CFB2046059956
:103830000A88CCE65E4815A90A4678C878C278C8D6
:1038400078C20125E8073A68136803431360B86833
:10385000FEF7B8FB02200026139C2168BA6AF965BE
:103860003A6610997966BE66F8660C980068129AF6
:103870001168091811600E9B19684A1C1A602268A9
:1038800010182060002900D0F6E41095384660300A
:1038900013903C465C3438460830129006210F984D
:1038A000FFF72EFC3868216881600C980068119041
:1038B00000F096FA04463868C069C00706D000F0E8
:1038C0008FFA001B149909888842F4D900F088FA0D
:1038D0000446109D3A68D069800707D500F080FA49
:1038E000001B149909888842F4D93A687420385C1E
:1038F00001282DD0E9042CE000F072FA0446386863
:10390000C069C00706D000F06BFA001B1499098843
:103910008842F4D900F064FA04463868C16989071E
:1039200007D500F05DFA001B149909888842F4D984
:1039300038680121029A11602249816100263046CF
:103940001DB0F0BD04210160002C00D191E491E490
:103950002905119C174B2340591801280C9D02D0B2
:103960001920400601E00720C00608181249401837
:103970005060002C0ED000F033FA04463A68D0694B
:10398000800707D400F02CFA001B1499098888429C
:10399000F4D93A682B681398016812980068074CAC
:1039A00000941432FEF77EFB30461DB0F0BDC046D9
:1039B00050E40202FF3F000000808000FDC20202CE
:1039C00068F60202000093EB10B501242046FEF7D2
:1039D00021FA204600F0DCF9002010BD124A072829
:1039E00009D880000F238340814019401068984314
:1039F0000843106070470F280AD8800020380F2332
:103A00008340814019405068984308435060704794
:103A1000800040380F2383408140194090689843CC
:103A2000084390607047C04634000040AEB0FEF7D7
:103A300075F8FEF7A8F8FEF7C1F80024204600F05C
:103A4000C9FDFFF7C1FFFEF79DF89A4806AD29466C
:103A5000CCC8CCC1CCC8CCC120462146FEF7F2FE72
:103A60002046294600F088FB93A0FDF751FA7D20FF
:103A70008000009001200290400603909748049037
:103A80009B4D9C4E05E0A6A0FDF7B0FA0398FCF70D
:103A90003FFE05A805800020FEF740FC0028FAD173
:103AA000002005AF02238F493A46FFF717F8388800
:103AB00030808949884232D18FA0FDF729FA0298D7
:103AC000020300273846874D2946FEF713FE05AC52
:103AD0000223384629462246FFF700F82088308026
:103AE0007D4988420CD119200203039C20467B4962
:103AF000FCF722FC206880F3088860680019804782
:103B000080A0FDF705FA23200203002738467349F9
:103B1000FEF7F0FDF0600028754D00D191E0002027
:103B200005AC02236E492246FEF7D8FF208870803C
:103B3000A84213D078498842A5D07849884213D04A
:103B400019200203039C20466449FCF7F5FB20681A
:103B500080F308886068001980479AE77CA0FDF729
:103B6000D7F9FDF743F994E771A0FDF73FFA192063
:103B7000020300205949FEF7BDFDFDF7D3FE029870
:103B8000C704704C1436704D002064233946224619
:103B9000FEF7A4FF0020FEF7C1FB0028FAD1204663
:103BA0003146FDF721FF204610303146FDF71CFF5E
:103BB000204620303146FDF717FF20463030314691
:103BC000FDF712FF204640303146FDF70DFF20463D
:103BD00050303146FDF708FF204660303146FDF792
:103BE00003FF0020642304992246FFF76BF90020AD
:103BF000FEF794FB0028FAD104986430049038460C
:103C00006430AF420746BFD305AC50482080002542
:103C100002262846324F39463246FEF76BFD2846CB
:103C2000394622463346FFF74DF90098FEF7B4F9BE
:103C3000BFF34F8F2C482D490860BFF34F8F00BF53
:103C4000FDE737614648B0803846019708E049A053
:103C5000FDF75EF93069401C3061B188884216DAA0
:103C6000B760C7013F4839180EAC802520462A4668
:103C7000FCF762FB19483918019F384622462B464B
:103C8000FFF7C4FAF0600028E1D137A0E0E70A208E
:103C9000FEF782F93A48FDF73BF90098FEF77CF908
:103CA000BFF34F8F104811490860BFF34F8F00BF1B
:103CB000FDE7C046B0E402024D4B383030302D42B3
:103CC0006F6F744C6F616465722D56312E30C6F47F
:103CD000B6AF0D0A00000000DDDD000000A000040A
:103CE00010D0020400F007040400FA050CED00E017
:103CF000AAAA000060EE0202BDF8C8EBB0E1D4CB86
:103D00000D0A0000B2C1B3FDB1EAD7A2CEBBB3C960
:103D1000B9A60D0A00000000CCCC0000BBBB00001F
:103D20004F5441C9FDBCB6C6F4B6AF0D0A00000041
:103D3000CDF8C2E7C9FDBCB6C6F4B6AFC6F4B6AF9F
:103D40000D0A0000E4F102029CFF0900FFFF0000E1
:103D5000B4AEBFDAC9FDBCB6C6F4B6AF0D0A0000FA
:103D60006104000000F0020474657374313D300D8D
:103D70000A00000074657374313D310D0A000000C3
:103D8000FFE50202014800687047C0460C00004091
:103D900001218140044A1F2802D010688843106026
:103DA00010680843106070471C000040004800473E
:103DB000C1A0020210B5401E07494860FF2000065E
:103DC000064A13688343032084071B1913600022EB
:103DD0008A60086010BDC04610E000E020ED00E001
:103DE00080B50020FEF786F9404280BDB0B586B0B0
:103DF000104869460A4638C838C238C838C2002454
:103E00002046FEF77DF903992046FEF7E1F9019877
:103E1000012803D00824002804D102E0042400284B
:103E200000D104460220FDF7FDFFE0400249086092
:103E300006B0B0BD0CE4020268F60202F0B583B031
:103E40000278CC48C36893421AD0446D944217D08C
:103E50008368934203D0046D944200D07EE09B1AA5
:103E60005A1E9341029348225A43032942D184188F
:103E7000E269002A4FD01C340020206003B0F0BD5E
:103E80009B1A5A1E9341029348225A43032916D182
:103E90008418A26B01920126EFF31085354002D100
:103EA000EFF3108772B6A76910229743A761A26942
:103EB000002A2BD0002D00D162B6019C0AE08218A6
:103EC00094691832302C02D01468102C01D180244F
:103ED0001460002448225A43801800228263026240
:103EE0008262243000220260002C37D002A8A04752
:103EF00003B0F0BD821894691832302C02D01468D7
:103F0000202C01D18024146000241BE0183426608A
:103F1000002DD1D0D1E7E26B01920126EFF310859D
:103F2000354002D1EFF3108272B6A2692027BA435E
:103F3000A261A269002A01D118342660002D00D1A7
:103F400062B6019C48225A4380180022C263C262B2
:103F50004263303000220260002CC7D103B0F0BDB4
:103F6000F0B583B0029048210A464243E04B9C588A
:103F7000E6690F2535409A18167C002E31D04F2067
:103F800040026169014200D185E0A06904218843B3
:103F9000A06102202062012081076918D161D36BE2
:103FA000EFF31084044002D1EFF3108572B69569E7
:103FB0002026B54395619569002D00D173E0104628
:103FC0003C30002C00D162B600240460D4625463FB
:103FD000303200201060002B63D002A8984703B055
:103FE000F0BD0C2D5DD8C0467D442D796D00AF44E9
:103FF0006358675806589DA1585858580600956947
:10400000202D04D0154618352D68302D49D1156B5B
:10401000566B3432AE4217D26669360714D56468DF
:1040200015686E1C166048431818C06A44550298FB
:104030000C4644431A19156B566B3432AE4203D208
:104040001C5966693607EAD41268AA4229D141434D
:10405000585882690524A24382615A18D36B012102
:10406000EFF31080084002D1EFF3108472B6946928
:104070002025AC4394619469002C02D11446183475
:10408000216014463C34002800D162B60021216032
:10409000D16251639CE70C2D00D176E7012D00D150
:1040A00073E703B0F0BD15461835286010463C3064
:1040B000002C00D187E787E70120206203B0F0BD24
:1040C00008252562164618369569102D02D03568E8
:1040D000302DE6D10196566A15462835976AB742C3
:1040E0002CD1A06902218843A061936B0121EFF3D9
:1040F0001080084002D1EFF3108472B6019E34683C
:104100001027BC4334603468002C00D13160144661
:104110003834002800D162B6002121602960116284
:10412000243200201060002BBBD056E70220206212
:1041300003B0F0BD0420206203B0F0BD2A68B24293
:10414000AFD262699207ACD52A68561C2E604843EC
:104150001818006A805C206002980A4642439D1845
:10416000AC6A6E6AB4429CD228359C586269920748
:10417000EAD496E748ED0202F0B585B00D46064652
:10418000022804D3002D02D1012005B0F0BD002E7D
:1041900003D0012E08D1092400E008242046FDF7B1
:1041A00039FE2046FFF7F4FD48217143504A50582C
:1041B00083691F240294A3438361062383600F2332
:1041C0000193036257180023BB62BB63FB633B622E
:1041D0007B62FB623B63297F39746A7F7A74AA7FB2
:1041E000BA7404937B636B68AA68EC6892002243FC
:1041F0005B1E032B0ED8C0467B441B795B009F449B
:1042000001030507082304E0182302E0282300E047
:1042100038231A43C260C907090F6A699201D2B2F2
:104220008918AA699207920E8918491C81607961E0
:104230002969012901D122210161384612300390F8
:104240000324002E01D0204600E0042029684C43BE
:1042500028490E19B178FDF76DFE3968CA688025C6
:1042600010462843C8602348005D73781B02181865
:10427000C862AA43CA60FDF796FE0398007800283A
:1042800009D1384611300078002804D13846103062
:104290000078002827D07868002815D4032102462A
:1042A0008A43164953588407E40EFF26A640B343B9
:1042B000A5401D4355500299014001208840D8492E
:1042C00008600F4908600EE08107C90EFF228A408E
:1042D000019C0440083C032084430748235893432F
:1042E0008D401D4325500120B861049805B0F0BDF4
:1042F00048ED020224E402021CED00E000E400E0CC
:1043000000E100E0F0B591B010900126002900D145
:104310009BE003930591002A00D196E007900121CC
:10432000EFF310800291084002D1EFF3108172B6D2
:1043300004924823069307994B43A449C9188D69F1
:104340000026302D6ED80C461834AD00374602A634
:1043500075593E46AF46C046F5E10202FDE1020254
:1043600001E2020201E2020201E2020201E20202B1
:1043700001E2020201E2020201E2020201E20202A1
:1043800001E2020201E2020201E2020201E2020291
:1043900001E2020201E20202E5E1020201E202029E
:1043A00001E2020201E2020201E2020201E2020271
:1043B00001E2020201E2020201E2020201E2020261
:1043C00001E2020201E2020201E2020201E2020251
:1043D00001E2020201E2020293E2020201E20202AF
:1043E00001E2020201E2020201E2020201E2020231
:1043F00001E2020201E2020201E2020201E2020221
:1044000001E2020201E2020201E2020201E2020210
:1044100001E2020201E20202E5E1020202260028B4
:104420000CD00CE0402D01D0802D05D101260028B4
:1044300004D004E010252560002800D162B6002ECB
:10444000069D624F049C079802D0304611B0F0BD23
:1044500000268E62039A8A63059A0A624C620A7C7D
:10446000002A0BD00C960B960A96099608960E9683
:1044700002220D9201282DD018202CE08A7C2831B0
:10448000002A3BD00A68A24216D22B464343FA5870
:104490005469A40710D50868441C0C60F918096A0F
:1044A000085C10601098294641437A18114628315B
:1044B000936A526A9342E8D34543785981698222CC
:1044C0000A438261304611B0F0BD302525600028D6
:1044D000B4D0B4E71A200F90C86808A9FDF772FDA0
:1044E000109845437A597819C0683949009105995F
:1044F0002346FDF7D7FD304611B0F0BDFB589A6951
:10450000140602D58024A2439A610A680026049802
:1045100082422ED25D694F225202154207980AD07C
:1045200002211962029EB10729431FE028315D690B
:1045300015423E46F4D137465C69A40702D4069979
:10454000224E0AE00C68661C0E60069948431F4E16
:104550003018006A005D1860109841437358711854
:104560008C6A4E6AB442E1D329463E46069D174FF7
:1045700001E0314607985A6A002AFCD1EFF3108215
:10458000029B1A4002D1EFF3108372B645437819AB
:1045900083691024A34383618369002B05D0002A1B
:1045A00009D0826B002A0BD14FE703461833029CD7
:1045B0001C60002AF5D162B6826B002A00D144E764
:1045C00010A89047304611B0F0BDC04648ED020239
:1045D00005DC0202B0B5002801D00120B0BD0320E7
:1045E00081020C4802680C4B535000249460012255
:1045F00053030A4D2B60BFF34F8FBFF36F8F084DEE
:104600002B6003685A50847204811020FDF7FAFB76
:104610002046B0BDD8ED020251E5CC1A80E100E0A1
:1046200080E200E002E008C8121F08C1002AFAD1A7
:1046300070477047002001E001C1121F002AFBD122
:1046400070470000000000000000000001000000B2
:10465000FFFFFFFF000000000000000059062014CB
:104660000321450128820032410032190041130024
:10467000390300B506002D03002D0200220100229F
:1046800001003E01002000000000000000000000CA
:104690000000000000000000000000000200000018
:1046A00000000000140000000200000007000000ED
:1046B00002000000020000000000000002000000F4
:1046C00000000000140000000200000001000000D3
:1046D00002000000020000000200000000000000D4
:1046E00014000000000000000700000000000000AF
:1046F00000000000030000000000000000000000B7
:1047000000000000010000000000000000000000A8
:104710000200000004000000001003EB0000000095
:104720000100000001000000040000000001003250
:104730000000000000000000000000000100000078
:104740000100000500000000000000000000000063
:104750000100000001000035000000000100000021
:104760000000000004000000000000200000000025
:10477000010000000000000004000000000000D85C
:104780000000000001000000000000000100000027
:104790000000000600000000010000000000000012
:1047A0000100000002000001000000000000000005
:1047B00000000000010000000300009F0000000056
:1047C000010000000000000001000000000000B92E
:1047D00000000000010000000000000001000000D7
:1047E000000000AB0A0A0D2050726F6772616D6D98
:1047F000696E6720436F6D706C65746564205375D6
:10480000636365737366756C6C79210A0D2D2D2DAC
:104810002D2D2D2D2D2D2D2D2D2D2D2D2D2D2D2DC8
:104820002D2D2D2D2D2D2D2D2D2D2D2D2D0D0A2008
:104830004E616D653A2000B0E1D4CBB3C9B9A6A3EF
:10484000ACD7BCB1B8D6D8C6F40D0A0034E6020223
:1048500000EC0202E801000048A1020288E6020220
:10486000E8ED0202840D0000FCE3020252033280F4
:1048700052014426B80303455006C570014013D6C3
:10488000207001401445B000500B4202820345FFE6
:10489000FF0F203204420832010456100001055176
:1048A0002000500745900140184204023D0545A0F4
:1048B0000140194206023D07454001400D820100BA
:1048C000FFFFFFFFFFFFFFFFFFFFFFFFFFFFFFFFF8
:1048D000FFFFFFFFFFFFFFFFFFFFFFFFFFFFFFFFE8
:1048E000FFFFFFFFFFFFFFFFFFFFFFFFFFFFFFFFD8
:1048F000FFFFFFFFFFFFFFFFFFFFFFFFFFFFFFFFC8
:10490000FFFFFFFFFFFFFFFFFFFFFFFFFFFFFFFFB7
:10491000FFFFFFFFFFFFFFFFFFFFFFFFFFFFFFFFA7
:10492000FFFFFFFFFFFFFFFFFFFFFFFFFFFFFFFF97
:10493000FFFFFFFFFFFFFFFFFFFFFFFFFFFFFFFF87
:10494000FFFFFFFFFFFFFFFFFFFFFFFFFFFFFFFF77
:10495000FFFFFFFFFFFFFFFFFFFFFFFFFFFFFFFF67
:10496000FFFFFFFFFFFFFFFFFFFFFFFFFFFFFFFF57
:10497000FFFFFFFFFFFFFFFFFFFFFFFFFFFFFFFF47
:10498000FFFFFFFFFFFFFFFFFFFFFFFFFFFFFFFF37
:10499000FFFFFFFFFFFFFFFFFFFFFFFFFFFFFFFF27
:1049A000FFFFFFFFFFFFFFFFFFFFFFFFFFFFFFFF17
:1049B000FFFFFFFFFFFFFFFFFFFFFFFFFFFFFFFF07
:1049C000FFFFFFFFFFFFFFFFFFFFFFFFFFFFFFFFF7
:1049D000FFFFFFFFFFFFFFFFFFFFFFFFFFFFFFFFE7
:1049E000FFFFFFFFFFFFFFFFFFFFFFFFFFFFFFFFD7
:1049F000FFFFFFFFFFFFFFFFFFFFFFFFFFFFFFFFC7
:104A0000FFFFFFFFFFFFFFFFFFFFFFFFFFFFFFFFB6
:104A1000FFFFFFFFFFFFFFFFFFFFFFFFFFFFFFFFA6
:104A2000FFFFFFFFFFFFFFFFFFFFFFFFFFFFFFFF96
:104A3000FFFFFFFFFFFFFFFFFFFFFFFFFFFFFFFF86
:104A4000FFFFFFFFFFFFFFFFFFFFFFFFFFFFFFFF76
:104A5000FFFFFFFFFFFFFFFFA5A54B4D000000106C
:104A600000000002AAAA5A7F20E80202000000000B
:104A70000200000000000000000000000000000034
:104A80000000000000000000000000000000000026
:104A90000000000000000000B8E802020000000072
:104AA0000A56656E646F72093A204D4B53454D4965
:104AB0000A43686970093A204D4B383030300A4457
:104AC000617465093A204A616E2020332032303209
:104AD000350A56657273696F6E093A2056302E3664
:104AE0002E32000000000000000000000000000066
:104AF000004B0000008000021400000018020000BB
:104B00000026B803004001400D0000000100000035
:044B100000000000A1
:020000040000FA
:104B2000A5A54B4D0000001000000002AAAA5A7F64
:104B3000204B000000000000020000000000000008
:104B40000000000000000000000000000000000065
:104B50000000000000000000000000000000000055
:104B6000B84B0000000000000A56656E646F7209C1
:104B70003A204D4B53454D490A43686970093A2024
:104B80004D4B383030300A44617465093A204A612F
:104B90006E20203320323032350A56657273696FC9
:104BA0006E093A2056302E362E32000000000000EA
:084BB0000000000000000000FD
:04000005000000C136
:00000001FF
